:100000000C949B040C94BA040C94B8040C94B8049B
:100010000C94B8040C94B8040C94B8040C94B80470
:100020000C94B8040C94B8040C94B8040C94B80460
:100030000C94B8040C94B8040C94B8040C94B80450
:100040000C94B8040C94B8040C94B8040C94B80440
:100050000C94B8040C94B8040C94B8040C94B80430
:100060000C94B8040C94B8046279204D696B652037
:10007000426172746F6E005858636F6E74726F6C69
:100080006C6572004553432063616C000000000002
:1000900000000000000000006779726F0061636378
:1000A000656C0098009D00526F6C6C005069746321
:1000B0006800A700AC004F66660042757A7A6572E8
:1000C000004C4544206C696768747300B600BA0040
:1000D000C10041DE008C008C008C001B190041EA3D
:1000E0000012018C00230116190041FB00DE008C78
:1000F0000045010000534554757000411201EA00AB
:100100008C000B060000444941476E6F73746963AD
:10011000730041DE00FB008C003A0800005265735A
:10012000657400418C008C00DE00390100004350F2
:10013000542F53772D56657200418C008C0023019B
:100140008C00E61600415C019E01EA00B901000046
:100150005345542F5478537469636B0041720145C1
:1001600001EA00EC0200005345542F53454E736FD3
:100170007200418B015C01EA0022040000534554E7
:100180002F43414D736572766F7300419E0172017A
:10019000EA00390500005345542F4C5641004145B3
:1001A000018B01EA00F30500005345542F4175749B
:1001B0006F2D44697361726D0041D5010B024501D9
:1001C000240200005345542F54782F43616C696218
:1001D000726174650041F001B9014501A203B413D5
:1001E0005345542F54782F5226502D526174650078
:1001F000410B02D5014501A203BB135345542F54B3
:10020000782F5961772D526174650041B901F00171
:1002100045013C0200005345542F54782F41726D24
:10022000696E6700418C008C00B9013002D4160061
:10023000418C008C00B9018C0000190041560271FC
:10024000020B028C0200005345542F54782F534167
:100250002F53696465004171023C020B02A4020045
:10026000005345542F54782F53412F506F696E74AB
:1002700000413C0256020B02C80200005345542FB5
:1002800054782F53412F44656C617900419802984E
:10029000023C028C00D5140041980298023C028C6A
:1002A00000E1140041BC02B00256028C00AC150003
:1002B00041BC02B00256028C00CD150041BC02B018
:1002C0000256028C00C1150041E002D40271028C7A
:1002D000006B150041E002D40271028C00A01500F1
:1002E00041E002D40271028C0094150041040350D5
:1002F000035C016A037D135345542F53454E2F521F
:100300006F6C6C00411D03EC025C016A03841353A3
:1003100045542F53454E2F50697463680041340390
:1003200004035C016A038C135345542F53454E2F2D
:10033000596177004150031D035C01A203F613537A
:1003400045542F53454E2F4163632D4761696E001D
:1003500041EC0234035C01C60300005345542F53A3
:10036000454E2F43616C69622E004286038603EC82
:1003700002A203C2135345542F53454E2F2E2E2F46
:100380004761696E5000426A036A03EC02A203CE21
:10039000135345542F53454E2F2E2E2F4761696E10
:1003A000490043BA03AE036A038C00B4180043BA91
:1003B00003AE036A038C00F2180043BA03AE036A6B
:1003C000038C00E4180041E203E2035003FE03DA69
:1003D000135345542F53454E2F2E2E2F43616C2D12
:1003E000470041C603C6035003FE03E113534554BF
:1003F0002F53454E2F2E2E2F43616C2D4100421658
:10040000040A04C6038C007B18004216040A04C6C2
:10041000038C00A618004216040A04C6038C00953B
:100420001800413C043C0472015604E8135345543F
:100430002F43414D2F536572766F310041220422C4
:100440000472015604EF135345542F43414D2F536B
:100450006572766F3200427104A6042204C1040062
:10046000005345542F43414D2F2E2E2F4178697351
:1004700000428B0456042204D90400005345542F33
:1004800043414D2F2E2E2F4469720042A604710461
:100490002204F10400005345542F43414D2F2E2ECA
:1004A0002F4761696E004256048B04220415050033
:1004B000005345542F43414D2F2E2E2F5472696DFA
:1004C0000042CD04CD0456048C004C150042CD04EE
:1004D000CD0456048C005C150042E504E50471046B
:1004E0008C002E150042E504E50471048C003D15D6
:1004F00000420905FD048B048C00891600420905A1
:10050000FD048B048C00C61600420905FD048B0413
:100510008C00B81600422D052105A6048C004A1651
:1005200000422D052105A6048C007B1600422D05F6
:100530002105A6048C006D16004152056C058B0147
:10054000870500005345542F4C56412F5365747551
:100550007000416C0539058B01AB055014534554AF
:100560002F4C56412F43616C69622E004139055270
:10057000058B01CF0500005345542F4C56412F4C9D
:100580006F774261747400419F05930539058C00B3
:10059000051500419F05930539058C002015004184
:1005A0009F05930539058C0012150041C305B70559
:1005B00052058C00FB150041C305B70552058C00A0
:1005C00073180041C305B70552058C006B18004134
:1005D000E705DB056C058C0028180041E705DB0505
:1005E0006C058C0061180041E705DB056C058C008B
:1005F00057180041FF05FF059E018C00EE140041D5
:10060000FF05FF059E018C00FA14004123064C06ED
:10061000FB0071065014444941472F53454E736FF8
:100620007273004136060B06FB001607501444494E
:1006300041472F527800414C062306FB0099075092
:1006400014444941472F4D6F746F7200410B0636B9
:1006500006FB0065065014444941472F4C6F6F70EC
:100660005261746500418C008C004C068C00681748
:1006700000418A06F0060B060A077D1344494147EC
:100680002F53454E2F526F6C6C0041A40671060B20
:10069000060A078413444941472F53454E2F50699A
:1006A0007463680041BC068A060B060A078C134473
:1006B0004941472F53454E2F5961770041D6068A4D
:1006C000060B060A079513444941472F53454E2F01
:1006D0004163632D580041F006BC060B060A079DD6
:1006E00013444941472F53454E2F4163632D590011
:1006F000417106D6060B060A07A513444941472F48
:1007000053454E2F4163632D5A00428C008C00717B
:10071000068C00BF1700412E07760723068D07FDC4
:1007200013444941472F52782F526F6C6C00414758
:1007300007160723068D070214444941472F5278B4
:100740002F506974636800415F072E0723068D07E9
:100750000814444941472F52782F436F6C6C004175
:100760007607470723068D070E14444941472F5249
:10077000782F596177004116075F0723068D07140C
:1007800014444941472F52782F41757800428C001C
:100790008C0016078C00FD160041B00714083606C1
:1007A0002E081A144D313A546F702D4C6566740042
:1007B00041C807990736062E0823144D323A546F64
:1007C000702D52696768740041DF07B00736062E46
:1007D000082C144D333A546F702D4261636B004105
:1007E000F907C80736062E0835144D343A426F749F
:1007F000746F6D2D4C65667400411408DF07360672
:100800002E083E144D353A426F74746F6D2D526947
:1008100067687400419907F90736062E0847144D9A
:10082000363A426F74746F6D2D4261636B00422ED5
:10083000082E0899078C00D91500418C008C0012F5
:10084000015208000052657365742F454550524FA0
:100850004D00418C008C0012015E08D01400411242
:1008600001120112011201A31400446F6E652100F0
:100870004E6F00205365636F6E64287329005961C1
:10088000772D5269676874005961772D4C656674DD
:1008900000755300487A202000203D00202D2000C4
:1008A000205B537461626C655D00205B4163726F15
:1008B0005D007553200044697361626C6564004596
:1008C0006E61626C6564004E6F7420417661696C84
:1008D00061626C65002025005265766572736564FF
:1008E000004E6F726D616C00446F6E652100526541
:1008F0006C6561736520537469636B732100536584
:100900007420436F6C6C2D3E4D696E00204C564137
:100910002050504D0056312E366A00436F6E74726F
:100920006F6C6C6572204572726F7200436F505429
:1009300065722059360011241FBECFEFD4E0DEBF10
:10094000CDBF11E0A0E0B1E0EAEDFAE302C005900E
:100950000D92AC30B107D9F712E0ACE0B1E001C0C4
:100960001D92A53AB107E1F70E940F130C946B1D7D
:100970000C9400001F920F920FB60F9211242F9328
:100980003F934F935F938F939F93EF93FF932091A8
:100990008400309185008091600190916101A901EE
:1009A000481B590B309361012093600183E1493862
:1009B000580718F01092620116C0909162019830A9
:1009C00090F4E92FF0E0E95DFD4FE2A9F0E0EE0FD1
:1009D000FF1FEB57FE4F5183408381E080939701C7
:1009E0009F5F90936201FF91EF919F918F915F9133
:1009F0004F913F912F910F900FBE0F901F90189520
:100A00004F925F926F927F928F929F92AF92BF921E
:100A1000CF92DF92EF92FF920F931F93CF93DF93CA
:100A2000782EE42F462E5524F0E0EE0FFF1FEB58F2
:100A3000FE4F60817181882777FD8095982F0E94F5
:100A4000BE1BF201EE0FFF1FEE0FFF1FEA53FE4F1A
:100A500020813181428153810E94721C0E948B1B34
:100A6000EB0160900E01662019F022E0721661F52C
:100A7000872D90E08C0163E0000F111F6A95E1F76C
:100A8000880F991F080F191F02531E4FBE01882798
:100A900077FD8095982F0E94BE1B9B01AC01D80169
:100AA00016966D917D918D919C9119970E94BA1A1D
:100AB0000E948B1BEB01B2E07B1619F4D095C19517
:100AC000DF4F8824992451C0E72DF0E08F01000FFB
:100AD000111F33E0EE0FFF1F3A95E1F7E00FF11F12
:100AE000E253FE4F66817781808591852AE939E955
:100AF00049E55FE30E94721C6B017C01CE01880F07
:100B0000991F8C0F9D1F65E070E00E94F51C8827DF
:100B100077FD8095982F0E94BE1B9B01AC01C701F9
:100B2000B6010E94BA1A0E948B1BEB01000F111F25
:100B30000E551E4F60913A0270E0882777FD809530
:100B4000982F0E94BE1BF801208131814281538180
:100B50000E94721C20E030E048E452E40E94231B13
:100B60000E948B1B4B01C60FD71F80919601A72CAB
:100B7000BB24882309F49DC0F501EE0FFF1FEA5A3C
:100B8000FE4F808191818C0F9D1F918380832AE38A
:100B9000893992071CF088E99AE305C08856954C7C
:100BA00024F488E695EC918380837501EE0CFF1C9C
:100BB000F3E1CF2EF2E0DF2ECE0CDF1CBE01882742
:100BC00077FD8095982F0E94BE1B8201000F111F98
:100BD000000F111FF801E15EFD4F2081318142813C
:100BE00053810E94721C0E948B1BD6016D937C93D3
:100BF000F701EA5AFE4F60817181882777FD809561
:100C0000982F0E94BE1B08561E4FF801208131818B
:100C1000428153810E94721C0E948B1B2EEA31E09C
:100C2000E20EF31ED7016D937C93B1E0B71508F483
:100C300056C06B1611F4C819D9098501000F111F90
:100C4000F801EA0DFB1DEE0FFF1FBF016A5B7E4F2F
:100C5000E85BFE4F80819181DB0115969C938E931A
:100C600014978D919C919183808398012E5A3E4FC9
:100C7000D9018D919C91AE01481B590BDB014D931D
:100C80005C93D901CD93DC930C541E4FDB01149679
:100C90008D919C91159720813181820F931F840F34
:100CA000951F65E070E00E94F51CF8017183608378
:100CB00016C0D501AA0FBB1FFD01EA5AFE4F1182D3
:100CC0001082FD01ED5EFD4F11821082FD01E255A3
:100CD000FE4F11821082AC54BE4F1D921C92E72D24
:100CE000F0E0EE0FFF1FDF01A255BE4FCF018D5E7A
:100CF0009D4F2D913C91DC018D919C91280F391FC6
:100D0000DF01AC54BE4F8D919C91280F391FE75ED7
:100D1000FD4F31832083DF91CF911F910F91FF9081
:100D2000EF90DF90CF90BF90AF909F908F907F908B
:100D30006F905F904F900895AF92BF92CF92DF92E5
:100D4000EF92FF920F931F93CF93DF935B01C82F16
:100D5000D0E08E01000F111F000F111F0A591D4F07
:100D600023E7C22ED12CFB01D182C082F801208161
:100D7000E22EFF24EE0CFF1CEE0CFF1C82EA91E039
:100D8000E80EF91EFE01EE0FFF1FEE0FFF1FE859E0
:100D9000FD4F608170E0882777FD8095982F0E9435
:100DA000BE1B20E030E040EA51E40E94231B2DEC02
:100DB0003CEC4CEC5EE30E94BB1AF70120813181D0
:100DC000428153810E94721C0E948B1BF801818119
:100DD000882331F46D587F4FF5017183608305C01E
:100DE000C61AD70AF501D182C082CC0FDD1FCC0F05
:100DF000DD1FC759DD4F2881332727FD3095F501C9
:100E000080819181820F931F91838083DF91CF91A5
:100E10001F910F91FF90EF90DF90CF90BF90AF9018
:100E200008958FE380937E0010927B000895809355
:100E30007C0086EC80937A0080917A0086FDFCCF5E
:100E40009091780080917900382F20E0290F311D92
:100E5000C90108957F928F929F92AF92BF92CF92D5
:100E6000DF92EF92FF920F931F93CF93DF93E82EC1
:100E700000E011E0CEECD1E0F80181918F010E94F9
:100E80001707998388832A96F1E006301F07A1F798
:100E9000EE2009F078C058E2852E52E0952ECEEC77
:100EA000D1E040E4A42E41E0B42E7724F401808107
:100EB000488159812A813B81882329F4421B530BA5
:100EC0005D834C8304C0241B350B3D832C83F1E0F0
:100ED000F715D8F0F501608171810C811D81600FDB
:100EE000711F882777FD8095982F0E94BE1B20E0F8
:100EF00030E040E05FE30E94721C6E837F8388874E
:100F00009987F5011183008330C0CC80DD80F2E049
:100F10007F1641F4B601882777FD8095982F0E94AF
:100F2000BE1B1FC06E817F818885998520E030E0DF
:100F300048E951E40E94721C7B018C01B6018827AC
:100F400077FD8095982F0E94BE1B9B01AC01C801C4
:100F5000B7010E94BB1A20E030E040EA51E40E9451
:100F6000231B6E837F8388879987739483E090E047
:100F7000880E991E2A96E2E0F0E0AE0EBF1EF6E063
:100F80007F1609F093CFDF91CF911F910F91FF90C2
:100F9000EF90DF90CF90BF90AF909F908F907F9019
:100FA0000895AF92BF92CF92DF92EF92FF920F938C
:100FB0001F93DF93CF93CDB7DEB72C970FB6F8947E
:100FC000DEBF0FBECDBF082F80E190E09A838983FA
:100FD0009C838B839E838D8398878F839A87898751
:100FE0009C878B8710E07E010894E11CF11CEDE0EA
:100FF000AE2EB12CAC0EBD1E7CE2C72E71E0D72EFA
:1010000081E00E942A07A701AEECB1E0F7018081E0
:1010100091812D913C911197820F931F8193919310
:101020001A96EA15FB0599F78AE392E0F6013197E3
:10103000F1F70197D9F72E9B02C02E9801C02E9A86
:101040001F5F1032E9F6013011F033E001C036E0E5
:10105000E0EDF1E020E0DA018D919D91AD0165E0D8
:10106000969587956A95E1F7918380832F5F3A96ED
:10107000231788F3013071F48091020290910302EA
:1010800020913D0230913E02821B930B909303020C
:101090008093020281E08093AA012E9A2C960FB6CB
:1010A000F894DEBF0FBECDBFCF91DF911F910F919E
:1010B000FF90EF90DF90CF90BF90AF900895809118
:1010C000790190917A0197FF8BC040917B015091FB
:1010D0007C018FEF413658070CF482C060910C01FF
:1010E000623009F47DC02091B20080915D01281B1F
:1010F00080915E0190915F01820F911D90935F013D
:1011000080935E018091B20080935D0180917002B6
:10111000681751F480916F0290E0909581959F4FF0
:10112000841795075CF406C080916F0290E0481721
:10113000590724F410925F0110925E0180917102B0
:1011400090E023EE36E1A901849F9001859F300D48
:10115000949F300D112480915E0190915F012817BA
:101160003907F0F580E0613009F081E080930C01EF
:101170008130B1F51092AA01809106010E94D10739
:101180001092060180918400909185009093A101B6
:101190008093A00180E090E0A0E0B0E08093C201E5
:1011A0009093C301A093C401B093C5018093BE0185
:1011B0009093BF01A093C001B093C1018093BA0185
:1011C0009093BB01A093BC01B093BD0188EC8093C8
:1011D000080110920F0180917902823009F45C9A23
:1011E000089580918400909185009093A10180934F
:1011F000A00180E090E0A0E0B0E08093C201909375
:10120000C301A093C401B093C5018093BE01909324
:10121000BF01A093C001B093C1018093BA01909324
:10122000BB01A093BC01B093BD0108955F926F9282
:101230007F928F929F92AF92BF92CF92DF92EF9266
:10124000FF920F931F93CF93DF937B018C013901A2
:101250004A010E94231B5B016C0120E030E048EC56
:1012600052E40E94721C9F770E948B1BEB01552455
:10127000C801B70120E030E040E050E00E941F1BB1
:10128000882314F455245394C436D1058CF52B9738
:10129000D4F0C601B50129E23CE54FE85EE30E94C7
:1012A000721CA60195010E94721C20E030E040E80B
:1012B0005FE30E94BB1A9B01AC01C601B5010E940D
:1012C000231B5B016C01C401B30120E030E040E06E
:1012D00050E00E941F1B88239CF5552039F5C6015C
:1012E000B5012BED3FE049E450E40E94BB1A26C053
:1012F000C601B501A60195010E94721C29E23CE5D8
:101300004FE85EE30E94BB1A9B01AC01C601B50128
:101310000E94231B9B01AC016BED7FE089EC9FE3F6
:101320000E94BA1A5B016C01552051F0C601B5014B
:101330002BED3FE049E450E40E94BA1A5B016C01D6
:10134000C601B50120EE3EE245E652E40E94721C61
:10135000DF91CF911F910F91FF90EF90DF90CF9091
:10136000BF90AF909F908F907F906F905F90089507
:101370002F923F924F925F926F927F928F929F92A5
:10138000AF92BF92CF92DF92EF92FF920F931F9393
:10139000DF93CF93CDB7DEB7A1970FB6F894DEBF3A
:1013A0000FBECDBF20918400309185008091A001B7
:1013B0009091A101B901681B790B3093A101209391
:1013C000A00180E090E00E94BC1B20916F01309151
:1013D000700140917101509172010E94231B6E8B2C
:1013E0007F8B888F998F6093240170932501809360
:1013F00026019093270120913D0230913E023D8BC2
:101400002C8BB901882777FD8095982F0E94BE1BF1
:10141000688B798B8A8B9B8B80917301909174017F
:1014200022273327281B390BB2ED2B2EB1E03B2EA0
:101430001B821A8241E0498344245524A90166276E
:1014400057FD6095762F4A8F5B8F6C8F7D8F9C0147
:10145000442737FD4095542F2E8F3F8F48A359A323
:1014600082010C5C1E4FD1016D917C91882777FD24
:101470008095982F0E94BE1B2E893F89488D598DDB
:101480000E94721CF8016083718382839383D1016F
:1014900090966D907D908D909C909397C401B30130
:1014A00020E030E040E251E40E94721C2889398932
:1014B0004A895B890E94231B7B018C01EA81FB81A5
:1014C000BF01882777FD8095982F0E94BE1B5B0186
:1014D0006C01C801B701A80197010E94721C9B0111
:1014E000AC01C601B5010E94BB1A0E948B1B7B8315
:1014F0006A839201285D3E4FF201E654FE4F8081DF
:101500009181A281B381F90180839183A283B38306
:10151000F6EE2F16F1E03F0659F16A8D7B8D8C8D2A
:101520009D8D0E94BE1B9B01AC01C401B3010E94B2
:101530001F1B87FD0EC06E8D7F8D88A199A10E9413
:10154000BE1B9B01AC01C401B3010E946E1C1816A6
:101550000CF419822AE030E0220E331E44E050E001
:10156000440E551E50EF251651E0350609F078CF90
:101570002090340130903501409036015090370171
:10158000609128017091290180912A0190912B018D
:101590006C877D878E879F87809138019091390174
:1015A000A0913A01B0913B0188879987AA87BB87B0
:1015B00020912C0130912D0140912E0150912F014D
:1015C0002C833D834E835F83C201B1012C853D8511
:1015D0004E855F850E94721C7B018C016885798530
:1015E0008A859B852C813D814E815F810E94721C82
:1015F0009B01AC01C801B7010E94BB1A9B01AC0161
:101600006091C2017091C3018091C4019091C501A4
:101610000E94BA1A6093C2017093C3018093C401FF
:101620009093C501A0903001B0903101C09032017B
:10163000D090330160903C0170903D0180903E015C
:1016400090903F01C201B101A60195010E94721C58
:101650007B018C01C401B3012C813D814E815F81EE
:101660000E94721C9B01AC01C801B7010E94BB1A09
:101670009B01AC016091BA017091BB018091BC01EA
:101680009091BD010E94BB1A6093BA017093BB0197
:101690008093BC019093BD01688579858A859B857F
:1016A000A60195010E94721C7B018C01C401B3014B
:1016B0002C853D854E855F850E94721C9B01AC0187
:1016C000C801B7010E94BA1A9B01AC016091BE012A
:1016D0007091BF018091C0019091C1010E94BB1A1D
:1016E0006093BE017093BF018093C0019093C101CC
:1016F0004A815B81455250404F39510578F4A2EF41
:101700008A2EA1E09A2EFAEB2F2EF1E03F2EAA248A
:101710006C897D892B016624772404C07981772325
:1017200071F734C0D401ED90FD900D911C91B2E0A1
:10173000AB1649F4E981EE2331F0C301B2010E94F6
:10174000BC1B7B018C01D1016D917D918D919C9190
:1017500020E030E847EC53E40E94721CA801970196
:101760000E94BB1A20E030E048EC53E40E94231BA7
:10177000F10161937193819391931F01A3942AE0E6
:1017800030E0820E931E33E0A31661F6E090C201B2
:10179000F090C3010091C4011091C5016091BA019C
:1017A0007091BB018091BC019091BD01A80197018E
:1017B0000E9416096093A2017093A3018093A40173
:1017C0009093A5016091BE017091BF018091C0010D
:1017D0009091C101A80197010E9416096093A6018A
:1017E0007093A7018093A8019093A901A1960FB6C9
:1017F000F894DEBF0FBECDBFCF91DF911F910F9147
:10180000FF90EF90DF90CF90BF90AF909F908F9020
:101810007F906F905F904F903F902F900895FF9230
:101820000F931F93CF93DF93F82E462FC62FD0E050
:10183000FE01EE0FFF1F8F010B571E4F10929701F5
:10184000D8018D919C91880F991F63E070E00E94F0
:10185000E11C80919701882389F7FF2029F0EB583C
:10186000FE4F718360833FC0CE0FDF1FC95DDD4F28
:10187000888D998D681B790B423039F4EB58FE4FF7
:10188000759567957595679529C0EB58FE4F44305F
:1018900061F471836083605971401CF410920E01F1
:1018A00022C081E080930E011EC0759567957595E5
:1018B00067957183608380916102282F30E08827CB
:1018C0009927821B930B861797071CF0620F731FD3
:1018D00005C0621773072CF0621B730B7183608362
:1018E00002C011821082DF91CF911F910F91FF9062
:1018F00008951F93182F60E00E940F0C812F61E064
:101900000E940F0C812F62E00E940F0C812F63E078
:101910000E940F0C812F64E00E940F0C1F9108950C
:101920000F931F93CF93DF93009184001091850054
:1019300010931A01009319012A9A299A289A5F9AFA
:101940005E9A5D9A80911B018F5F80931B018630A8
:1019500071F410921B01599A2F9A80E06CE072E0AA
:101960000E949C0681E06EE072E00E949C06ACE161
:10197000B1E0CEE1D1E020E080E090E03CEDFC0180
:10198000ED59FE4F0190F081E02DED3DF10514F091
:10199000388301C0E883223080F4FC01E45FFD4F0E
:1019A0000190F081E02DF7FF02C01C9206C0ED3DD2
:1019B000F10514F03C9301C0EC932F5F0296119651
:1019C00021962630E1F680E00E942A070000000000
:1019D00000000000F8948091840090918500801BA5
:1019E000910B789425E0803A920780F39093180148
:1019F00080931701A89816BCF0911E01E0911F0179
:101A000070912001609121015091220140912301A8
:101A100030911C0120911D0190E09F1709F42A9834
:101A20009E1709F42998971709F42898961709F42E
:101A30005F98951709F45E98941709F45D989317C9
:101A400009F45998921729F42F9803C00000000058
:101A5000000086B58D32D0F386B58D5286BD9F5F6E
:101A60009D3DD9F6DF91CF911F910F910895CF93AE
:101A7000DF9380910A0190910B01009711F001977B
:101A800009C080910C01813019F48CE291E002C010
:101A900088EB91E090930B0180930A0180910A01F9
:101AA00090910B01892B09F05BC080910F01882375
:101AB00071F010920F018BB182958F7080958170BB
:101AC0008295807F9BB19F7E982B9BB949C086E011
:101AD0000E941707AC019093AC018093AB018091F9
:101AE00079028823B1F020910701222321F481E0BB
:101AF00080930F010EC080910A0290910B0284170F
:101B0000950720F021502093070103C085E08093C2
:101B1000070180917302882319F1809108018823BD
:101B200021F481E080930F011BC080917901909195
:101B30007A01181619061CF488EC8093080190911C
:101B40000C01913069F480910801882349F081509B
:101B500080930801882321F410920C0190930F01C7
:101B6000109296018091790190917A014A971CF028
:101B700081E08093960180910C01813019F080E022
:101B80000E942A070E94B80980E060E040E00E94BD
:101B9000000581E060E041E00E94000582E061E034
:101BA00043E00E940005C0917901D0917A01C43CC4
:101BB000D10514F0C3ECD0E0D0937A01C093790141
:101BC00080E009C0E82FF0E0EE0FFF1FED59FE4F57
:101BD000D183C0838F5F8630A8F380911D029091DE
:101BE0001E02833391051CF082E390E005C08E5CF9
:101BF0009F4F34F48EEC9FEF90931E0280931D0252
:101C00002091190230911A02C901B3E0880F991F7F
:101C1000BA95E1F7821B930B68E070E00E94F51C17
:101C2000AB0170931A026093190260911B027091CC
:101C30001C02E0911D02F0911E02809167019091BB
:101C40006801860F971F8E1B9F0B909368018093EE
:101C50006701CF01860F971F20916D0130916E01B2
:101C6000820F931F90936E0180936D017595679518
:101C700070931C0260931B02809163019091640138
:101C8000841B950B861B970B8E1B9F0B90936401F7
:101C9000809363019F01261B370B8091690190910E
:101CA0006A01841B950B280F391F30936A0120931A
:101CB000690180916501909166018E1B9F0B840FD5
:101CC000951F861B970B9093660180936501461BB9
:101CD000570B80916B0190916C01480F591F4E0F6B
:101CE0005F1F50936C0140936B0120E049E150E08D
:101CF0000DC0E22FF0E0EE0FFF1FED59FE4F808187
:101D00009181499714F4518340832F5F263088F3E3
:101D100020935C011C161D0624F48091AA018823DF
:101D200079F480E009C0E82FF0E0EE0FFF1FED59D5
:101D3000FE4F118210828F5F8630A8F380935C0182
:101D400080910C01813011F40E94900CDF91CF91B1
:101D50000895AF92BF92CF92DF92EF92FF921F93BE
:101D6000DF93CF93CDB7DEB728970FB6F894DEBFD9
:101D70000FBECDBF1A8219821C821B821E821D8259
:101D800018861F8210E05CE2C52E51E0D52E7E0140
:101D90000894E11CF11C49E0A42EB12CAC0EBD1E30
:101DA00025C0F6013197F1F70197D9F72E9881E018
:101DB0000E94790C8EE091E0F6013197F1F70197DE
:101DC000D9F7B70145E751E0F70180819181DA0148
:101DD0002D913D91AD01820F931F81939193AE168A
:101DE000BF0699F72E9A1F5F103119F086E292E034
:101DF000D8CFEFE3F2E0DB018D919D91BD0134E09E
:101E0000969587953A95E1F7918380833396AA1644
:101E1000BB0689F78D819E8124E0969587952A954A
:101E2000E1F70E96909346028093450228960FB6EE
:101E3000F894DEBF0FBECDBFCF91DF911F91FF9011
:101E4000EF90DF90CF90BF90AF90089582EE94E036
:101E50002CE231E0F9013197F1F70197D9F72E9A89
:101E600082EE94E02CE231E0F9013197F1F701972D
:101E7000D9F72E9808951F93CF93DF93EC01162F77
:101E80000E94551D811721F0CE01612F0E945D1D1A
:101E9000DF91CF911F910895CF92DF92EF92FF9241
:101EA0000F931F93CF93DF938C016B017A01809185
:101EB00010028093660080E69AEE0197F1F7C0E089
:101EC000D0E009C0C6018C0F9D1FF80161918F0100
:101ED0000E943B0F2196CE15DF05A0F3809195015E
:101EE0008093660088E99AE30197F1F7DF91CF913B
:101EF0001F910F91FF90EF90DF90CF90089587E2B0
:101F000092E062E370E043E550E00E944C0F0895D8
:101F1000AF92BF92CF92DF92EF92FF920F931F93F7
:101F20000E947F0F6091620270E080E090E00E946A
:101F3000BC1B20E030E042E852E40E94231B5B011E
:101F40006C0160931F027093200280932102909392
:101F500022026091630270E080E090E00E94BC1B6E
:101F600020E030E543E456E40E94231B609398018F
:101F70007093990180939A0190939B016091640200
:101F800070E080E090E00E94BC1B20E030E04AEF6F
:101F900052E40E94231B7B018C0160932302709307
:101FA000240280932502909326026091650270E0DE
:101FB00080E090E00E94BC1B20E030E543E456E462
:101FC0000E94231B60939C0170939D0180939E014E
:101FD00090939F016091570270E080E090E00E9432
:101FE000BC1B20E030E044EB52E40E94231BA6011E
:101FF00095010E94231B6093C6017093C7018093D3
:10200000C8019093C9016091580270E080E090E0AF
:102010000E94BC1B20E030E042E852E40E94231BF7
:10202000A80197010E94231B6093CA017093CB0102
:102030008093CC019093CD0160913B0270913C0262
:1020400080E090E00E94BC1B20E030E44CE156E4CC
:102050000E94721C60936F017093700180937101F4
:102060009093720160913D0270913E0280E090E099
:102070000E94BC1B2DE33AE047ED5EE30E94721C18
:102080000E948B1B709374016093730160917802BE
:1020900070E080E090E00E94BC1B209174023091BF
:1020A000750240917602509177020E94721C0E9444
:1020B000901B70930B0260930A021F910F91FF9087
:1020C000EF90DF90CF90BF90AF900895E7E2F2E0FD
:1020D00083E5DF011D928A95E9F780E4809327026A
:1020E00081E08093280280932B0280932E0210922D
:1020F00031028093340210923702789680EF95E097
:102100001282918380833396B2E0E735FB07C1F7F3
:1021100080E694E090934602809345023C9788EED7
:1021200093E0128291838083339622E0E735F207B1
:10213000C1F780E090E0FC01E95DFD4F82AB0196C4
:1021400088309105C1F782E08093610282E294E2D7
:1021500090933C0280933B0286E790E090933E028E
:1021600080933D0285E28093620282E38093630262
:1021700022E82093640284E68093650296E49093BB
:102180003A028FE5809357022093580290936F0292
:1021900091E09093700283E0809371021092660246
:1021A0008EE18093680290936A0280936C02109291
:1021B000790283E29BEDA9E7B0E4809374029093E7
:1021C0007502A0937602B093770289E68093780235
:1021D0000E947F0F089582E390E00E94551D803495
:1021E00019F00E946610089587E292E062E370E0C1
:1021F00043E550E00E94451D089580911601882313
:10220000C1F481E080931601109212021092110223
:102210001092AD0187E790E00E94C91988E690E02E
:102220000E94E71980E00E94790C8AEB80931401E8
:102230001BC08230C9F483E08093160189EC99E1D8
:10224000909386028093850280910C01823029F45C
:1022500082ED90E00E94741307C08EED90E00E9422
:10226000741381E00E94D1078091B2009091100117
:10227000891B2091110130911201280F311D3093DB
:102280001201209311018091B2008093100127392F
:10229000310508F477C0265930403093120120935D
:1022A000110180E00E94790C2E9880910C01882306
:1022B00041F4809113018F5F80931301815009F4E1
:1022C0002E9A809114018F5F8093140189320CF44F
:1022D00052C0109214018091AD01882329F0E09141
:1022E0001102F0911202099580911601883018F4BC
:1022F0008F5F809316012091790130917A01213A04
:102300003105A4F180910901882381F10E94260FF3
:102310000E94260F81E00E94D10710920601809151
:102320008400909185009093A1018093A00180E0AA
:1023300090E0A0E0B0E08093C2019093C301A0932D
:10234000C401B093C5018093BE019093BF01A093D7
:10235000C001B093C1018093BA019093BB01A093D7
:10236000BC01B093BD011092090105C037FF03C045
:1023700081E08093090180911501882319F0815033
:102380008093150180911501882309F042C0809146
:102390001601843008F43DC0809177019091780156
:1023A0002FEF8D3D920744F4E0918302F091840277
:1023B00033968591949119C0849744F0E0918302FB
:1023C000F09184023196859194910FC080917501AE
:1023D000909176012FEF8D3D92076CF4E09183028E
:1023E000F09184023596859194910E94281386E29B
:1023F000809315010895849764F0E0918302F09131
:1024000084023796859194910E94281386E28093E6
:10241000150108950F931F93CF93DF9388E893E1FD
:102420002CE231E0F9013197F1F70197D9F780916A
:10243000660080939501809310020E94EB1020911A
:1024400066008AEE91E0821B910965E070E00E94CF
:10245000F51C80916600AB01480F511D4F3F51059F
:1024600019F014F08FEF03C080916600860F8093FF
:1024700095018091100287FD07C08091950187FF2B
:1024800003C08A51809395018091950180936600E5
:1024900085B7806185BF52983A98399838983B98AB
:1024A0003C983D98229A219A209A579A569A559A82
:1024B000519A279A269A2E98549A5C9883E0809392
:1024C000690081E08DBB8CBB14BC85BD10926E0091
:1024D0001092800082E0809381001092B00087E02B
:1024E0008093B1001092700017BA1092B20086E18A
:1024F0000E946A198FE380937E0010927B001092F5
:10250000AA011092970178945C9A0E94260F5C9819
:1025100081E00E942A0781E00E942A0780E29EE46F
:102520002CE231E0F9013197F1F70197D9F7EEECA0
:10253000F1E020E0808191818C529140815991405D
:1025400048F082E080930C01233008F481E080930E
:102550000D0104C02F5F3A96253061F780E00E949C
:10256000790C8091790190917A01813A91050CF46E
:1025700048C084E890E00E94C9191092680082E087
:102580008CBB0CED10E0C0EFD2ED80E00E94790C26
:102590008091790190917A01499690937A01809384
:1025A00079018D3D91052CF010937A01009379010A
:1025B00006C0499724F410927A0110927901809113
:1025C000790190917A0190936401809363019093D3
:1025D00066018093650190936801809367019093F1
:1025E0006A018093690190936C0180936B019093D1
:1025F0006E0180936D010E94900CCE010197F1F75E
:10260000C4CF1092960180917902823009F45C9ACD
:102610000E94880FDF91CF911F910F9108950E9422
:102620000A1280E00E94790C0E945F0880910C01E0
:10263000823011F00E94370D80910C01813089F3B6
:102640000E94FD10EECFFC01009709F00995089556
:102650009C0180E02C38380709F445C0F9019491B9
:102660004091830250918402FA018491981798F462
:10267000E0917A02E150E0937A02FF27E7FDF095BE
:10268000EE0FFF1FE558FD4F8081918190938402EA
:102690008093830215C0891778F480917A02E82F1D
:1026A000FF27E7FDF095EE0FFF1FE558FD4F408334
:1026B00051838F5F80937A02309384022093830248
:1026C0008091830290918402E0918502F0918602CC
:1026D0000B960995E0918302F091840239968591D9
:1026E00094910E942313089510927A029093840289
:1026F000809383020E942813089510929D021092E5
:102700009E021092AD01089581E080939D02109287
:102710009E021092AD01089582E080939D0281E0B7
:1027200080939E021092AD01089583E080939D02F4
:1027300010929E021092AD01089584E080939D0254
:1027400010929E021092AD01089585E080939D0243
:1027500010929E021092AD01089588E492E0909349
:102760009A0280939902089587E592E09093A002DF
:1027700080939F02089588E592E09093A002809351
:102780009F02089580919E0290E0880F991F8E59B4
:102790009D4F9093A00280939F02089580919E0286
:1027A00090E0880F991F8D599D4F9093A0028093C0
:1027B0009F0208958BE392E09093A4028093A3027A
:1027C00008958DE392E09093A4028093A30208956C
:1027D00086E692E090939C0280939B0208958AE69D
:1027E00092E090939C0280939B0208958AE392E08A
:1027F0009093A00280939F0208951092AD011092D1
:102800009D0208951092AD0181E080939D0208958C
:102810001092AD0182E080939D0208951092AD0167
:1028200083E080939D0208951092AD0184E080932F
:102830009D02089583E691E09093A2028093A10205
:102840001092AD01089585E691E09093A2028093E5
:10285000A1021092AD01089587E691E09093A20243
:102860008093A1021092AD01089589E691E09093C2
:10287000A2028093A1021092AD0108958BE691E02F
:102880009093A2028093A1021092AD0108958DE66B
:1028900091E09093A2028093A1021092AD0108955D
:1028A0001092AD0108956091AB017091AC0180E090
:1028B00090E00E94BC1B20917402309175024091FF
:1028C0007602509177020E94231B20E030E040E81E
:1028D0005EE30E94BB1A0E94901BDC01CB010895AD
:1028E000DF92EF92FF920F931F93182F0E945314C1
:1028F0001B3219F4D82ED39402C0D82EDA946091EA
:10290000AB017091AC0180E090E00E94BC1B7B01A8
:102910008C016D2D70E080E090E00E94BC1B9B015B
:10292000AC01C801B7010E94231B6093740270932D
:10293000750280937602909377021F910F91FF901A
:10294000EF90DF900895DF93CF93CDB7DEB7289750
:102950000FB6F894DEBF0FBECDBFDE011196E9E5DC
:10296000F2E088E001900D928150E1F70E9466103C
:10297000A9E5B2E0FE01319688E001900D92815008
:10298000E1F70E947F0F8AE698E00E94E7192896F7
:102990000FB6F894DEBF0FBECDBFCF91DF91089583
:1029A00080E798E00E94E7190895809170028823DB
:1029B00019F488E898E002C08EE798E00E94E719D1
:1029C000089590E080917002882309F491E090933B
:1029D00070020E94D5140E947F0F089580917302A7
:1029E000882319F08FEB98E002C086EB98E00E94F4
:1029F000E71908958091730291E08927809373020B
:102A00000E94EE140E947F0F089580917902E82FB2
:102A1000F0E0EE0FFF1FE453FF4F859194910E9469
:102A2000E719089580917902882311F482E001C0AA
:102A30008150809379020E9405150E947F0F0895AE
:102A4000809179028F5F80937902833011F4109224
:102A500079020E9405150E947F0F0895E0919B0264
:102A6000F0919C028181882319F481EE98E002C0E4
:102A700088ED98E00E94E7190895E0919B02F0919B
:102A80009C0290E08181882309F491E091830E9467
:102A90002E150E947F0F0895E0919B02F0919C02F9
:102AA0008081E82FF0E0EE0FFF1FEE54FF4F85917D
:102AB00094910E94E7190895E0919B02F0919C0285
:102AC00090E08081882309F491E090830E944C1566
:102AD0000E947F0F089587E892E00E94B31A6091E8
:102AE0007102669587E892E070E041E021E00E9483
:102AF000FB1987E892E06EE20E948F1A80917102C2
:102B000080FD02C060E301C065E387E892E00E94B7
:102B10008F1A87E892E063E778E00E949D1A87E8C1
:102B200092E00E94B619089580917102823018F0E7
:102B30008150809371020E946B150E947F0F08954F
:102B4000809171028A3018F48F5F809371020E9425
:102B50006B150E947F0F08950F931F9307E812E0F3
:102B6000C8010E94B31A60916F02C80170E042E090
:102B700021E00E94FB19C8010E94B6191F910F9114
:102B8000089580916F02893218F0815080936F020E
:102B90000E947F0F0E94AC15089580916F028A35C4
:102BA00018F48F5F80936F020E947F0F0E94AC1514
:102BB00008958091AD01882349F489ED95E19093C2
:102BC00012028093110281E08093AD0187E892E0C8
:102BD0000E94B31AE091A102F091A202608171817A
:102BE00087E892E041E022E00E94FB1987E892E04A
:102BF0000E94B61908951F938091AD01882349F46E
:102C000081E08093AD018BEF95E190931202809368
:102C1000110287E892E00E94B31A8091AB01909173
:102C2000AC018837910538F487E892E067EC78E0EA
:102C30000E949D1A24C00E945314182F6AE00E941B
:102C4000D51C682F87E892E070E042E021E00E9406
:102C5000FB1987E892E06EE20E948F1A812F6AE0EA
:102C60000E94D51C692F87E892E070E041E021E0E6
:102C70000E94FB1987E892E066E50E948F1A809116
:102C80007902882309F45C9887E892E00E94B619DB
:102C90001F91089587E892E00E94B31AE0919B0289
:102CA000F0919C02838118162CF487E892E06BE285
:102CB0000E948F1AE0919B02F0919C02638177271A
:102CC00067FD709587E892E041E021E00E94FB19E2
:102CD00087E892E00E94B6190895E0919B02F09176
:102CE0009C028381833E14F0815083830E944A16A4
:102CF0000E947F0F0895E0919B02F0919C028381D6
:102D00008E3114F48F5F83830E944A160E947F0FD6
:102D1000089587E892E00E94B31AE0919B02F09137
:102D20009C026281669587E892E070E042E021E0D3
:102D30000E94FB1987E892E06EE20E948F1AE091F0
:102D40009B02F0919C02828180FD02C060E301C081
:102D500065E387E892E00E948F1A87E892E065EDCC
:102D600078E00E949D1A87E892E00E94B6190895C3
:102D7000E0919B02F0919C028281853010F081509D
:102D800082830E9489160E947F0F0895E0919B0222
:102D9000F0919C0282818A3F10F48F5F82830E94AF
:102DA00089160E947F0F08950F931F9307E812E082
:102DB000C8010E94B31AC8016EEF78E00E949D1A04
:102DC000C8010E94B6191F910F9108950F931F9388
:102DD00007E812E0C8010E94B31AC80165E179E072
:102DE0000E949D1AC8016CE079E00E949D1AC801FA
:102DF0000E94B6191F910F9108950F931F93809110
:102E0000AD01882349F481E08093AD018DEF96E117
:102E10009093120280931102E0919D02F0E0EE0F78
:102E2000FF1FEB57FE4F80819181880F991F63E050
:102E300070E00E94E11C162F072F80E00E94790CA1
:102E400087E892E00E94B31A87E892E0612F702F22
:102E500044E021E00E94FB1987E892E062EB78E011
:102E60000E949D1A80919D028430D0F487E892E000
:102E70006BE50E948F1AE0919D02F0E0EE0FFF1FBC
:102E8000EB58FE4F6081718187E892E043E021E0DA
:102E90000E94FB1987E892E06DE50E948F1A11C02D
:102EA000843079F480910E01882329F487E892E038
:102EB0006AEA78E004C087E892E060EA78E00E947D
:102EC0009D1A87E892E00E94B6191F910F9108950C
:102ED0000F931F938091AD01882349F488E697E111
:102EE000909312028093110281E08093AD010091D2
:102EF00084001091850080E00E94790C0E945F0898
:102F00000E94370D8091840090918500801B910B69
:102F1000880F991F63E070E00E94E11C8B01085844
:102F20001A4F87E892E00E94B31A980140E050E0FF
:102F300060E472E48FE090E00E94081D87E892E070
:102F4000B90141E021E00E94FB1987E892E064E9C1
:102F500078E00E949D1A87E892E0B80141E021E004
:102F60000E94FB1987E892E061E978E00E949D1ACF
:102F700087E892E00E94B6191F910F910895809101
:102F8000AD01882349F48FEB97E19093120280936F
:102F9000110281E08093AD0180E00E942A0787E85A
:102FA00092E00E94B31A80919D0290E0FC0173E0D0
:102FB000EE0FFF1F7A95E1F7880F991FE80FF91FB1
:102FC000E253FE4F6081718187E892E044E021E0A6
:102FD0000E94FB1987E892E06CE978E00E949D1A54
:102FE00080919D0290E0FC01EE0FFF1FEE0FFF1F8E
:102FF000E80FF91FEE0FFF1FE053FE4F6081718154
:1030000087E892E043E021E00E94FB1987E892E024
:1030100069E978E00E949D1A80919D0290E0FC0190
:1030200033E0EE0FFF1F3A95E1F7880F991FE80F85
:10303000F91FE253FE4F6481758187E892E043E017
:1030400021E00E94FB1987E892E00E94B6190895DA
:103050000F931F9307E812E0C8010E94B31A8091F2
:1030600078026AE00E94D51C682FC80170E042E037
:1030700021E00E94FB19C8016EE20E948F1A809124
:1030800078026AE00E94D51C692FC80170E041E017
:1030900021E00E94FB19C80166E50E948F1AC80151
:1030A0000E94B6190E94880F1F910F910895809178
:1030B00078028D3318F08150809378020E9428188E
:1030C000089580917802803A18F48F5F8093780297
:1030D0000E94281808958DE20E9470140E94FB152A
:1030E0000E94880F08958BE20E9470140E94FB15C5
:1030F0000E94880F08950F931F9307E812E0C801FC
:103100000E94B31AE091A302F091A4026081718140
:10311000C80141E021E00E94FB19C8010E94B619D4
:103120000E94880F1F910F910895E091A302F091E2
:10313000A402808191818B30910518F002979183D0
:1031400080830E947B180E947F0F0895E091A30264
:10315000F091A402808191810296918380830E94E4
:103160007B180E947F0F089587E892E00E94B31AAF
:10317000E0919F02F091A0026081669587E892E05D
:1031800070E041E021E00E94FB1987E892E06EE2E6
:103190000E948F1AE0919F02F091A002808180FD31
:1031A00002C060E301C065E387E892E00E948F1AE5
:1031B00087E892E065E20E948F1A87E892E00E9419
:1031C000B6190E94880F0895E0919F02F091A00225
:1031D0008081853010F0815080830E94B4180E9455
:1031E0007F0F0895E0919F02F091A00280818A3FB5
:1031F00010F48F5F80830E94B4180E947F0F08959F
:103200008EEE98E00E94E71988E99AE32CE231E01B
:10321000F9013197F1F70197D9F70E94A90E88EECD
:1032200098E00E94E7190E947F0F08958CE299E0D0
:103230000E94C919089580910D018823B9F08BE18E
:1032400099E00E94C91920910D0181E090E0821B54
:103250009109880F991FEE27FF27E81BF90BED5501
:10326000FF4F859194910E94E71908958EED90E0AB
:103270000E9428130895582F2C9882E391E001971B
:10328000F1F741E020E030E062E371E0842F852334
:1032900011F02C9A01C02C98CB010197F1F7440F43
:1032A0002F5F3F4F2830310589F72C9A82E391E058
:1032B0000197F1F708951F93182F8CE70E943B198F
:1032C000812F80580E943B1988E99AE30197F1F712
:1032D0001F9108951F93182F249A2C9A8EEF0E9405
:1032E0003B19812F0E945B191F9108951F93182F7E
:1032F000803130F48EEF0E943B19812F805809C035
:10330000803210F010E0F6CF8EEF0E943B19812F33
:1033100080550E943B191F9108951F93813011F42D
:1033200080E003C0823051F480E10E94761910E001
:1033300080E20E943B191F5F1031D1F71F91089561
:10334000CF93DF93EC0182E00E948D1981E00E940F
:103350008D1980E00E94761903C021960E943B19C6
:1033600088818823D1F7DF91CF910895CF93DF93A0
:10337000EC0182E00E948D1980E10E94761903C061
:1033800021960E943B1988818823D1F7DF91CF9144
:1033900008951F93CF93DF93EC0182E00E948D1973
:1033A000FE011491112379F0219681E00E948D197C
:1033B00080E00E947619812F0E943B19FE01219620
:1033C00014911123C1F7DF91CF911F910895CF93ED
:1033D000DF93EC0182E00E948D1980E10E94761952
:1033E00002C00E943B19FE01219684918823C9F7EF
:1033F000DF91CF9108959F92AF92BF92CF92DF92CB
:10340000EF92FF920F931F93CF93DF93EC018B0109
:10341000C42ED22E77FD03C045E020E005C01095F4
:1034200001951F4F46E021E060E1E62E67E2F62EAF
:1034300030E050E2952E90E3A92E8DE2B82E0FC019
:10344000C801B7010E94E11C6E9DC0016F9D900DE7
:103450007E9D900D1124081B190B41507F013323D1
:1034600029F40E151F0510F4C416D0F1222381F0A3
:103470000E151F0518F482E0D81651F489898031A1
:1034800030F4FE01E80FF11DB0828F5F898B20E0E0
:10349000332319F40E151F0580F03989303158F4A3
:1034A000FE01E30FF11DC801B7010E94E11C605D40
:1034B00060833F5F398B31E013C0898992E0D91670
:1034C00039F4803168F4FE01E80FF11DA08206C0D6
:1034D000803130F4FE01E80FF11D90828F5F898BFF
:1034E000C7016AE070E00E94E11CFB0161307105D8
:1034F00031F481E0D81609F0A3CF31E0A1CF6115F6
:10350000710509F09DCFDF91CF911F910F91FF9031
:10351000EF90DF90CF90BF90AF909F900895DC0127
:1035200051968C915197803138F4FD01E80FF11DCF
:1035300060838F5F51968C930895DC010DC0519686
:103540008C915197803140F4FD01E80FF11D90837B
:103550008F5F51968C935197FB016F5F7F4F9491D2
:10356000992369F70895FC01118A81E111928A95E6
:10357000E9F708955058BB27AA270ED075C166D128
:1035800030F06BD120F031F49F3F11F41EF45BC199
:103590000EF4E095E7FB51C1E92F77D180F3BA171C
:1035A000620773078407950718F071F49EF58FC1C1
:1035B0000EF4E0950B2EBA2FA02D0B01B90190014E
:1035C0000C01CA01A0011124FF27591B99F0593F92
:1035D00050F4503E68F11A16F040A22F232F342FDA
:1035E0004427585FF3CF469537952795A795F04028
:1035F0005395C9F77EF41F16BA0B620B730B840B3D
:10360000BAF09150A1F0FF0FBB1F661F771F881FF4
:10361000C2F70EC0BA0F621F731F841F48F487954C
:1036200077956795B795F7959E3F08F0B3CF93953B
:10363000880F08F09927EE0F979587950895D9D0B0
:1036400008F481E008950CD00FC107D140F0FED0FE
:1036500030F021F45F3F19F0F0C0511139C1F3C0CF
:1036600014D198F39923C9F35523B1F3951B550B46
:10367000BB27AA2762177307840738F09F5F5F4F45
:10368000220F331F441FAA1FA9F333D00E2E3AF086
:10369000E0E830D091505040E695001CCAF729D0A0
:1036A000FE2F27D0660F771F881FBB1F26173707EF
:1036B0004807AB07B0E809F0BB0B802DBF01FF271F
:1036C00093585F4F2AF09E3F510568F0B6C000C185
:1036D0005F3FECF3983EDCF3869577956795B79559
:1036E000F7959F5FC9F7880F911D9695879597F974
:1036F0000895E1E0660F771F881FBB1F62177307ED
:103700008407BA0720F0621B730B840BBA0BEE1F01
:1037100088F7E095089504D06894B111D9C0089550
:10372000BCD088F09F5790F0B92F9927B751A0F0DF
:10373000D1F0660F771F881F991F1AF0BA95C9F745
:1037400012C0B13081F0C3D0B1E00895C0C0672F7E
:10375000782F8827B85F39F0B93FCCF386957795F5
:103760006795B395D9F73EF49095809570956195DE
:103770007F4F8F4F9F4F0895E89409C097FB3EF409
:1037800090958095709561957F4F8F4F9F4F9923AE
:10379000A9F0F92F96E9BB279395F695879577952C
:1037A0006795B795F111F8CFFAF4BB0F11F460FFEC
:1037B0001BC06F5F7F4F8F4F9F4F16C0882311F044
:1037C00096E911C0772321F09EE8872F762F05C058
:1037D000662371F096E8862F70E060E02AF09A95F3
:1037E000660F771F881FDAF7880F9695879597F9E8
:1037F0000895990F0008550FAA0BE0E8FEEF161682
:103800001706E807F907C0F012161306E407F507D4
:1038100098F0621B730B840B950B39F40A2661F048
:10382000232B242B252B21F408950A2609F4A140EB
:10383000A6958FEF811D811D089597F99F6780E8F8
:1038400070E060E008959FEF80EC089500240A94F2
:103850001616170618060906089500240A9412166B
:103860001306140605060895092E0394000C11F49E
:10387000882352F0BB0F40F4BF2B11F460FF04C04B
:103880006F5F7F4F8F4F9F4F089557FD9058440FA4
:10389000551F59F05F3F71F04795880F97FB991FAF
:1038A00061F09F3F79F0879508951216130614066C
:1038B000551FF2CF4695F1DF08C0161617061806F9
:1038C000991FF1CF86957105610508940895E894D4
:1038D000BB2766277727CB0197F908958ADF08F47D
:1038E0008FEF08950BD0C0CFB1DF28F0B6DF18F00E
:1038F000952309F0A2CFA7CF1124EACFC6DFA0F30A
:10390000959FD1F3950F50E0551F629FF001729F74
:10391000BB27F00DB11D639FAA27F00DB11DAA1F93
:10392000649F6627B00DA11D661F829F2227B00DE0
:10393000A11D621F739FB00DA11D621F839FA00D6B
:10394000611D221F749F3327A00D611D231F849FBB
:10395000600D211D822F762F6A2F11249F57504012
:103960008AF0E1F088234AF0EE0FFF1FBB1F661FAD
:10397000771F881F91505040A9F79E3F510570F066
:103980005CCFA6CF5F3FECF3983EDCF3869577954E
:103990006795B795F795E7959F5FC1F7FE2B880F61
:1039A000911D9695879597F90895991B79E004C024
:1039B000991F961708F0961B881F7A95C9F780956E
:1039C0000895AA1BBB1B51E107C0AA1FBB1FA61766
:1039D000B70710F0A61BB70B881F991F5A95A9F7B8
:1039E00080959095BC01CD01089597FB092E07267F
:1039F0000AD077FD04D0E5DF06D000201AF47095D8
:103A000061957F4F0895F6F7909581959F4F0895A2
:103A100097FB092E05260ED057FD04D014D00AD0EE
:103A2000001C38F450954095309521953F4F4F4FED
:103A30005F4F0895F6F790958095709561957F4F4B
:103A40008F4F9F4F0895A1E21A2EAA1BBB1BFD01A9
:103A50000DC0AA1FBB1FEE1FFF1FA217B307E4076D
:103A6000F50720F0A21BB30BE40BF50B661F771FC5
:103A7000881F991F1A9469F76095709580959095A5
:103A80009B01AC01BD01CF010895DC01CB01FC011C
:103A9000F999FECF06C0F2BDE1BDF89A319600B4A7
:103AA0000D9241505040B8F70895F999FECF92BD5C
:103AB00081BDF89A992780B50895262FF999FECFF0
:103AC0001FBA92BD81BD20BD0FB6F894FA9AF99A3B
:0A3AD0000FBE01960895F894FFCF91
:0C3ADA000201000304050105C8012000E2
:00000001FF
